:020000020000FC
:1000000027C018E01A95F1F708950AE03095089492
:1000100010F4C29A02C0C2980000F3DFF2DF3695F6
:100020000A95B1F7089509E0B19BFECFEADFE9DF59
:10003000E8DF8894B19B08940A9511F04795F7CFB3
:1000400008951FEF2AE02A95F1F71A95D9F7089538
:1000500010E820E016BD26BD11E01EBF1FE51DBF44
:10006000C29ABA9A3C9A3F9A3E983B983A9A399AE1
:10007000389A3D9A379A3598329A319830981AE2E0
:1000800023E3277F12601160106810641F7D1F7EBC
:100090002B7F2D7F21601ABD23BFB89A369AB5DF1A
:0A00A0003699FECF35B139BDF9CF16
:00000001FF
